:100000000C94D2040C9433050C94F8200C94330512
:100010000C9433050C9433050C9433050C94330580
:100020000C9433050C9433050C9433050C943C1D4F
:100030000C9433050C94131D0C9433050C94330568
:100040000C9433050C9433050C9433050C94ED1C7F
:100050000C9433050C9433050C9433050C94330540
:100060000C9433050C9433050C9433050C94330530
:100070000C9433050631FF0974A10109751500269A
:10008000FF009520750881020976150026FF00956E
:100090002075089102C005010902A1010901A10012
:1000A0008501050919012908150025019508750123
:1000B00081020501093009311581257F95027508F6
:1000C000810609381581257F950175088106050C83
:1000D0000A38021581257F950175088106C0C00583
:1000E000010980A10185021601002637001A81004E
:1000F0002AB700751095018100C0050C0901A10106
:100100008503160100269C021A01002A9C02751024
:1001100095018100C005010906A101050719E02923
:10012000E715002501950875018102950175088183
:1001300001050819012905950575019102950175BB
:100140000391010507190029FF150026FF009506F8
:1001500075088100C0722530325820007325303276
:100160005820005B6D253032642C253032645D20D0
:10017000005B6B253032585D200041726368696D09
:1001800065646573207374617274732E0A00255858
:100190003A253031366225730A000A202030313288
:1001A000333435363738394142434445460A005BDB
:1001B0004C45443A253032583A253032585D2000BB
:1001C0004C45443A20253032580A000A4C6F6F7073
:1001D0002073746172742E0A000A55534220636FB3
:1001E0006E666967757265642E0A000A544D4B3A53
:1001F0003565386139362F4C5546413A643661379A
:1002000064660A0009025400030100A032090400D8
:100210000001030101000921110100012240000732
:1002200005810308000A0904010001030102000915
:100230002111010001227F00070582030800010946
:100240000402000103000000092111010001222223
:1002500000070583032000011201100100000008BF
:10026000EDFEACAC0001010200013C034100720054
:100270006300680069006D0065006400650073003C
:1002800020006B006500790062006F006100720061
:100290006400200063006F006E007600650072004D
:1002A0007400650072000000080354004D004B000C
:1002B0000000040309046D6F7573653A205B2530F7
:1002C00032587C25642025642025642025645D0A3D
:1002D0000073797374656D3A20253034580A0063D1
:1002E0006F6E73756D65723A20253034580A003F81
:1002F000004D3E2000433E20000A00257500363A9E
:1003000020776865656C5F74696D655F746F5F6D9C
:1003100061783A20000A00257500353A2077686533
:10032000656C5F6D61785F73706565643A20000A83
:1003300000257500343A2074696D655F746F5F6DD8
:1003400061783A20000A00257500333A206D617803
:100350005F73706565643A20000A00257500323AC3
:1003600020696E74657276616C286D73293A20007D
:100370000A00257500313A2064656C6179282A31BC
:10038000306D73293A20000A092D2056616C75657D
:1003900073202D0A004D3E004D25643E20003F0095
:1003A0007365742064656661756C740A00433E2051
:1003B000000A002530325820006B6579626F617247
:1003C000643A2000293A3B3C3D3E3F404142434491
:1003D00045464748351E1F20212223242526272D48
:1003E0002E742A494A4B535455672B141A08151773
:1003F0001C180C12132F30314C4D4E5F6061567833
:10040000041607090A0B0D0E0F3334285C5D5E5786
:1004100079641D1B06190511103637387D52595A5B
:100420005B397A2C7E7C50514F626358808080808B
:1004300080808080808080808080808080808080BC
:1004400080808080290A002575002F002575005DB9
:100450002800256400200025640020002564002079
:10046000002564007C0025303258006D6F7573657F
:100470006B6579205B62746E7C78207920762068C9
:100480005D287265702F61636C293A205B000A0950
:100490002D204D61676963202D0A643A0964656205
:1004A00075670A783A096465627567206D617472D0
:1004B00069780A6B3A096465627567206B657962D1
:1004C0006F6172640A6D3A096465627567206D6FC9
:1004D0007573650A763A0976657273696F6E0A7389
:1004E0003A097374617475730A633A09636F6E73C2
:1004F0006F6C65206D6F64650A302D343A096C614C
:10050000796572302D34284631302D4634290A5011
:100510006175733A09626F6F746C6F616465720A1A
:10052000000A092D20436F6E736F6C65202D0A45FC
:1005300053432F713A09717569740A6D3A096D6FE9
:100540007573656B65790A003F0074696D65725F4C
:1005500072656164333228293A202530346C580A98
:10056000006B6579626F6172645F69646C653A20E3
:1005700025580A006B6579626F6172645F70726FF3
:10058000746F636F6C3A2025580A00686F73745F4C
:100590006B6579626F6172645F6C65647328293A78
:1005A0002025580A000A092D2053746174757320A0
:1005B0002D0A004743433A20372E332E3020415630
:1005C000522D4C4942433A20322E302E3020415693
:1005D000525F415243483A2061767233350A004FE8
:1005E0005054494F4E533A204C554641204D4F559B
:1005F00053454B45592045585452414B455920438A
:100600004F4E534F4C4520434F4D4D414E44204B90
:1006100045594D41505F53454354494F4E20424F39
:100620004F544C4F414445525F53495A450A00428A
:1006300055494C443A2035653861393620283132E5
:100640003A34383A3334204F637420333120323017
:100650003233290A005649443A2030784645454409
:1006600028544D4B29205049443A20307841434189
:10067000432841726368696D65646573206B6579B1
:10068000626F61726420636F6E7665727465722941
:10069000205645523A203078303130300A004445F7
:1006A00053433A20636F6E766572747320417263B0
:1006B00068696D65646573206B6579626F617264EA
:1006C00020696E746F205553420A000A092D205686
:1006D000657273696F6E202D0A000A6D6F75736500
:1006E0003A206F66660A000A6D6F7573653A206F6F
:1006F0006E0A000A6B6579626F6172643A206F66F8
:10070000660A000A6B6579626F6172643A206F6EE7
:100710000A000A6D61747269783A206F66660A0091
:100720000A6D61747269783A206F6E0A000A646516
:100730006275673A206F6E0A000A64656275673AEF
:10074000206F66660A000A0A626F6F746C6F6164DC
:1007500065722E2E2E2000433E20006D6B5F776861
:1007600065656C5F74696D655F746F5F6D6178203E
:100770003D2025640A006D6B5F776865656C5F6D71
:1007800061785F7370656564203D2025640A006DA3
:100790006B5F74696D655F746F5F6D6178203D207C
:1007A00025640A006D6B5F6D61785F7370656564C9
:1007B000203D2025640A006D6B5F696E746572765A
:1007C000616C203D2025640A006D6B5F64656C617F
:1007D00079203D2025640A006D6B5F776865656C44
:1007E0005F74696D655F746F5F6D6178203D202572
:1007F000640A006D6B5F776865656C5F6D61785F3B
:100800007370656564203D2025640A006D6B5F741C
:10081000696D655F746F5F6D6178203D2025640AA6
:10082000006D6B5F6D61785F7370656564203D205E
:1008300025640A006D6B5F696E74657276616C2069
:100840003D2025640A006D6B5F64656C6179203D15
:100850002025640A0077686572652064656C7461A0
:100860003A20637572736F723D25642C207768653A
:10087000656C3D25640A53656520687474703A2F71
:100880002F656E2E77696B6970656469612E6F7272
:10089000672F77696B692F4D6F7573655F6B65792E
:1008A000730A000A092D204D6F7573656B657920F9
:1008B0002D0A4553432F713A09717569740A313A0B
:1008C0000964656C6179282A31306D73290A323ADE
:1008D00009696E74657276616C286D73290A333A02
:1008E000096D61785F73706565640A343A097469EB
:1008F0006D655F746F5F6D61780A353A0977686579
:10090000656C5F6D61785F73706565640A363A097E
:10091000776865656C5F74696D655F746F5F6D6145
:10092000780A0A703A097072696E742076616C7583
:1009300065730A643A097365742064656661756C51
:1009400074730A75703A092B310A646F776E3A092D
:100950002D310A706775703A092B31300A7067645F
:100960006F776E3A092D31300A0A7370656564201D
:100970003D2064656C7461202A206D61785F73701E
:10098000656564202A2028726570656174202F20B7
:1009900074696D655F746F5F6D6178290A004C251D
:1009A000640A000011241FBECFEFD4E0DEBFCDBF2C
:1009B00004B603FE41C08091E1039091E203A0914F
:1009C000E303B091E4038730904BA740B04BA1F50F
:1009D0001092E1031092E2031092E3031092E403F9
:1009E00014BE0FB6F894A89580916000886180933A
:1009F0006000109260000FBE109201081092000873
:100A000089E0E3E0F0E080935700E491E695E3703D
:100A1000E15080E090E1E33040F4F0E0EE0FFF1FA2
:100A2000EE5CFE4F8081918100C0E0E0F0E8E81BC1
:100A3000F90BF695E795099511E0A0E0B1E0EAE63B
:100A4000F5E402C005900D92A833B107D9F723E071
:100A5000A8E3B1E001C01D92A13EB207E1F70E94F8
:100A60000F1E0C94B3220C940000FF93EF93E091BF
:100A70003801F0913901309709F00995EF91FF9114
:100A80000895FC018591803011F0EFDFFBCF0895D0
:100A9000FF27E0E230E247FF0CC0419597FF09C015
:100AA000EDE26095709580959095611D711D811D99
:100AB000911D27FF02C0219530E350E2AA27660F5F
:100AC000771F881F991FAA1FA41710F0A41B6395F6
:100AD0005A95A9F7AA3008F0A95FA05DAF93F395E6
:100AE000611571058105910541F7ED3211F4EF9320
:100AF000F395F21718F43F93F395FBCF8F91B5DF81
:100B0000FA95E1F70895E991F9918591803021F006
:100B1000853219F0AADFF9CF089520E0E8945591C5
:100B20005532C1F3503311F4689455915A3348F457
:100B3000505390F3220F022E220F220F200D250F6B
:100B4000F4CF0EF4219589919991533619F35337C7
:100B500029F1533559F1BC0188279927E8945C366F
:100B600021F48991999168945591543639F446EF5E
:100B70007EF077FF0DC08FEF9FEF0AC055374AE038
:100B800039F0583540E121F0523642E009F008953D
:100B9000FF93EF937DDFEF91FF91B7CFFF93EF933B
:100BA000FC0181918030B9F360DFFBCFFF93EF93BD
:100BB00068DFF1CFDF93CF93CDB7DEB72596A3DF04
:100BC000CF91DF910895803FC1F48091D30387FDD9
:100BD0001092D3038091D20381110EC08091D30370
:100BE00081110AC08091D403811106C08091D50380
:100BF000811102C01092CE030895813F29F48091A3
:100C0000D30318162CF3E6CF9091D203823F29F438
:100C100097FFE0CF1092D203DDCF833F19F419166E
:100C2000CCF3D8CF893F39F48091D403181694F6C9
:100C30001092D403CFCF8A3F29F48091D40387FF49
:100C4000C9CFF6CF8B3F39F48091D50387FFC2CF50
:100C50001092D503BFCF8C3F29F48091D50318168D
:100C6000BCF3B8CF843F31F48091D1038E7F809361
:100C7000D103B0CF853F21F48091D1038D7FF7CF91
:100C8000863F21F48091D1038B7FF1CF873F21F400
:100C90008091D103877FEBCF883F21F48091D103EE
:100CA0008F7EE5CF8D3F31F48091CD038E7F809391
:100CB000CD0390CF8E3F21F48091CD038D7FF7CF70
:100CC0008F3F09F087CF8091CD038B7FF0CF80914C
:100CD000CD0380FF0CC06091130170E0759567959E
:100CE000759567956115710559F1862F089581FFF6
:100CF00006C06091130170E075956795F3CF609120
:100D0000130170E082FD0CC06091CE036623A9F050
:100D1000209112018091130190E0621730F0BC0124
:100D200060387105F8F28FE7089570E00E94742230
:100D3000622F70E00E948522F3CF61E070E0D5CF92
:100D400081E008958091CD0380FF11C0809115014D
:100D500090E065E070E00E947422959587959595E6
:100D6000879580389105B0F50097B1F1089581FF1E
:100D70000AC08091150190E065E070E00E94742245
:100D800095958795EECF82FF08C08091150190E080
:100D900065E070E00E947422E4CF3091CE033323EB
:100DA000B1F0209114018091150190E065E070E0B0
:100DB0000E947422BC013217A0F6832F90E00E949B
:100DC0007422622F70E00E948522CB01CACF85E099
:100DD00090E008958FE7089581E00895803F31F411
:100DE0000E94A20681958093D3030895813F19F450
:100DF0000E94A206F8CF823F31F40E94A20681959C
:100E00008093D2030895833F19F40E94A206F8CF7D
:100E1000893F29F40E9467068093D40308958A3F8E
:100E200021F40E9467068195F7CF8B3F31F40E9431
:100E3000670681958093D50308958C3F19F40E942D
:100E40006706F8CF843F31F48091D10381608093AD
:100E5000D1030895853F21F48091D1038260F7CFBB
:100E6000863F21F48091D1038460F1CF873F21F444
:100E70008091D1038860EBCF883F21F48091D1032A
:100E80008061E5CF8D3F31F48091CD038160809307
:100E9000CD0308958E3F21F48091CD038260F7CF7A
:100EA0008F3FB9F78091CD038460F1CFE72FF0E059
:100EB00094E0EE0FFF1F9A95E1F7E60FF11DEC535A
:100EC000FC4F6491E62FE295E77090E023E0880FF5
:100ED000991F2A95E1F78E0F911D34E0880F991F15
:100EE0003A95E1F7E62FEF70E80FF92FF11DEE0FBD
:100EF000FF1FE050F8498591949108952FB7F89419
:100F00008091D6039091D703A091D803B091D903D3
:100F10002FBF0895829590E09C01220F331F220F6E
:100F2000331F2C7C95958795959587958373282BF2
:100F300030E0C901880F991F8A7A35952795257564
:100F4000822B08954F925F926F927F929F92AF9201
:100F5000BF92CF92DF92EF92FF920F931F93CF93A6
:100F6000DF9300D000D01F92CDB7DEB76B837C83B8
:100F70008D837A018C819D81892B49F08FEFF81246
:100F800004C081E09FEF491719F080E001C081E0C3
:100F900080FD6AC00F2D10E0CE2CD12C8B818823D0
:100FA00009F456C0409043035090440360904503B9
:100FB000709046038091DD039091DE03A091DF03E2
:100FC000B091E003482A592A6A2A7B2A2FE1A22EEF
:100FD000B12C9A2CD301C2010A2C04C0B695A79556
:100FE000979587950A94D2F780FD2BC081E0A81AC7
:100FF000B10878F7912CF80194E0EE0FFF1F9A9555
:10100000E1F7E95BFC4FEC0DFD1D9082E982FA826D
:1010100069817A81892D0F900F900F900F900F901A
:10102000DF91CF911F910F91FF90EF90DF90CF90C4
:10103000BF90AF909F907F906F905F904F900C9477
:101040005607B7018A2D0E945607019779F2D3CF30
:10105000F80184E0EE0FFF1F8A95E1F7E95BFC4F92
:10106000EC0DFD1D9080D2CF90E080E00F900F90AE
:101070000F900F900F90DF91CF911F910F91FF90E4
:10108000EF90DF90CF90BF90AF909F907F906F9048
:101090005F904F90089541E050E060E070E004C040
:1010A000440F551F661F771F8A95D2F740955095BC
:1010B000609570958091430390914403A0914503FE
:1010C000B091460384239523A623B723809343033B
:1010D00090934403A0934503B0934603089541E0E1
:1010E00050E060E070E004C0440F551F661F771F9A
:1010F0008A95D2F78091430390914403A0914503D0
:10110000B0914603842B952BA62BB72B80934303DA
:1011100090934403A0934503B093460308958091B0
:10112000420390911103981301C008958F5F877057
:10113000FACF1F93CF93DF9300D000D01F92CDB78B
:10114000DEB7942F4983252F5A836B837C838D834D
:101150004C815D8181E0452B31F02F3F19F481E016
:101160009F3F09F080E0182F117080FD2CC049814D
:101170005A816B817C818D810E94A207292F229543
:101180002F702C3078F42A30A8F422502230C8F086
:10119000812F0F900F900F900F900F90DF91CF91B4
:1011A0001F9108952C3011F02F3091F793FB1127E8
:1011B00010F9EECF803C28F0803E50F3815F833001
:1011C00038F311E0E5CF10E0E3CFE091C703F091F1
:1011D000C803309721F00190F081E02D099480E060
:1011E00008951092E2001092E100E0EEF0E08081BC
:1011F00081608083E8EDF0E080818F77808319BC87
:10120000E3E6F0E08081816080831092EF02089530
:101210000E94F108F89487E797E79093010880937C
:10122000000887E090EBDC018093E1039093E203F8
:10123000A093E303B093E40388E19CE00FB6F89435
:10124000A895809360000FBE90936000FFCFFC01D3
:10125000809103039091040386179707A0F061150E
:10126000710529F49091E8009E779093E80090E052
:101270006115710551F4911108C08091E80082FF59
:1012800032C080E00895BC01F2CF8091050388232D
:10129000B1F18530B1F18091E80083FD2EC08091DD
:1012A000E80082FDEACF8091E80080FFE1CF209145
:1012B000F20030E06115710519F02830310558F061
:1012C00091E02830310509F090E02091E8002E7778
:1012D0002093E800CDCF81918093F1006150710996
:1012E0002F5F3F4FE7CF80910503882341F0853082
:1012F00041F08091E80083FFC0CF81E0089582E053
:10130000089583E008952091E4003091E50085E69A
:101310009091EC0090FF06C09091E80090FF06C00D
:1013200080E008959091E80092FDFACF9091050336
:10133000992391F0953091F09091EB0095FD10C0BC
:101340004091E4005091E5002417350709F38150DE
:101350009A01F1F684E0089582E0089583E008950B
:1013600081E008958091FD0287FF13C08091E8001D
:1013700082FF06C08091E8008B778093E80004C06C
:10138000809105038111F2CF089580910503882390
:10139000D9F38091E80080FFF8CF8091E8008E7744
:1013A000ECCF982F9093E900242F762F50E08917E7
:1013B00031F07091EC002091ED005091F00021FD92
:1013C00007C09F5F953071F78093E90081E0089531
:1013D0003091EB003E7F3093EB003091ED003D7F8C
:1013E0003093ED003091EB0031603093EB0070935F
:1013F000EC002093ED005093F0002091EE0027FDCB
:10140000E0CF80E008950F931F93CF93DF93CDB784
:10141000DEB7AA970FB6F894DEBF0FBECDBF80919E
:101420000503882309F44EC11091E9001F708091D3
:10143000EC0080FF39C080E8182B1092E900809101
:10144000E80083FF3CC1EDEFF2E085E093E02091FE
:10145000F10021938E179F07D1F78091FE02833010
:1014600009F470C018F5813009F447C0823009F4DE
:10147000DAC08091E80083FF14C18091FD02909151
:10148000FE029A3008F00DC1E92FF0E0E65BF54F5F
:101490000C949922240B4A0B510B4A0B510BAC0BA9
:1014A000CE0B510BC90CD60C80E0C6CF8A3009F4A4
:1014B000A9C08B3009F47DC08930D9F68091FD0236
:1014C0008132B9F68091010390910203892B89F64C
:1014D0008091E800877F8093E8008091E80082FF98
:1014E0002CC08091F1008093F1028091E8008B770D
:1014F0008093E8000E94B209BCCF8091FD02813A3E
:1015000009F0B7CF8091E800877F8093E800809151
:10151000010390910203892B61F060E090E080E08C
:1015200070E00E9427098091E8008B778093E800A3
:10153000A0CF68E082EF92E0F3CF809105038111A4
:10154000CCCF97CF8091FD02813A09F092CF809164
:10155000010390910203892BA1F48091E800877F19
:101560008093E8008091E80080FFFCCF809111011A
:101570008093F1008091E8008E778093E8000E94CC
:10158000B2098091010390910203019709F071CF94
:101590008091E800877F8093E8008091E80080FFD9
:1015A000FCCF809110018093F1008091E8008E774C
:1015B0009FCF8091FD02813209F05BCF80910103C2
:1015C00090910203892B59F48091E800877F8093E2
:1015D000E8000E94B2098091FF028093110180917E
:1015E000010390910203019709F043CF8091E80035
:1015F000877F8093E8000E94B2098091FF02809368
:10160000100137CF8091FD02813209F032CF8091F5
:10161000E800877F8093E8000E94B2098091000370
:101620008093DA0326CF8091FD02813A09F021CF21
:101630008091E800877F8093E8008091E80080FF38
:10164000FCCF8091DA03AFCF803889F0823849F53A
:10165000809101038F70853020F58093E90080919F
:10166000EB0085FB882780F91092E90006C0809185
:10167000FA029091FB02911182609091E800977FAD
:101680009093E8008093F1001092F1008091E800BF
:101690008E7731C0282F2D7F21F48823F1F08230FE
:1016A00079F18091E80083FF0AC08091E800877F8C
:1016B0008093E8008091EB0080628093EB001F70C4
:1016C0001093E900AA960FB6F894DEBF0FBECDBF07
:1016D000DF91CF911F910F9108958091FF0281308A
:1016E00001F7933009F080E08093FB021092E9004B
:1016F0008091E800877F8093E8000E94B209D1CFF3
:101700008091FF028111F2CF809101038F702FEF42
:10171000280F243030F68093E9002091EB0020FF61
:10172000E5CF933031F48091EB0080628093EB0041
:10173000DDCF9091EB0090619093EB0021E030E0E1
:1017400001C0220F8A95EAF72093EA001092EA007E
:101750008091EB008860EACF8111A3CF0091FF0256
:101760000F778091E3008078802B8093E300809155
:10177000E800877F8093E8000E94B2098091E8002A
:1017800080FFFCCF8091E30080688093E30083E0DA
:10179000011101C082E08093050383CF805882301D
:1017A00008F07FCF2091FF02309100032C3D83E0B1
:1017B0003807A1F583E08A838AE289834FB7F894DA
:1017C000DE01139620E03EE051E2E32FF0E050937B
:1017D0005700E49120FF03C0E295EF703F5FEF7088
:1017E0008E2F90E0EA30C0F0C7968D939D932F5FC7
:1017F000243159F74FBF8091E800877F8093E8003C
:101800006AE270E0CE0101960E9427098091E8000B
:101810008B778093E80045CFC096E7CF8091010396
:1018200090910203432F55274330510509F44FC0CF
:1018300078F54130510509F445C084E590E0E4E0D5
:10184000F2E04230510509F02CCF2091E800277FCB
:101850002093E8002091030330910403821793073B
:1018600008F49C0140E02115310509F063C04111E5
:1018700061C08091E80082FDC9CF80910503882373
:1018800029F2853019F28091E80083FFF2CFBECFB4
:101890004132510509F43FC04232510509F001CFF0
:1018A0008330910508F0FDCEFC01EE0FFF1FE45ED2
:1018B000FE4F0190F081E02D875E9E4FDC018C9100
:1018C00090E01DC082E190E0E8E5F2E0BECF332772
:1018D00021303105C1F060F02230310509F0E1CE50
:1018E000EAE6F2E0E4918E2F90E0EAE6F2E007C04B
:1018F000E2EBF2E0E4918E2F90E0E2EBF2E0009771
:1019000009F4CFCEA2CFE8EAF2E0E4918E2F90E086
:10191000E8EAF2E0F4CF8330910508F0C2CE880FF8
:10192000991FFC01EE5DFE4F0190F081E02D89E0F2
:1019300090E08BCF80910503882309F467CF853031
:1019400009F464CF8091E80083FD60CF8091E800C6
:1019500082FD8FCF8091E80080FF85CF8091F200DB
:1019600090E02115310519F08830910550F041E0E3
:10197000089709F040E08091E8008E778093E800B6
:1019800072CF44914093F100319621503109019674
:10199000E8CF803809F085CE8091E800877F80937A
:1019A000E8008091FC028093F10070CE811179CE25
:1019B0000091FF02023008F074CE8091E800877F2A
:1019C0008093E8000093FC020E94B209002399F082
:1019D00084E08093050342E061EC81E00E94D1093C
:1019E00042E061EC82E00E94D10946E261EC83E0D2
:1019F0000E94D10956CE8091E30087FDE9CF81E0B6
:101A0000E8CFEF92FF920F931F93CF937C018B014E
:101A10000E948309C82F811119C08091E80085FDBB
:101A20000DC08091E8008E778093E8000E94030A41
:101A30000E948309882389F3C82F08C0F701819188
:101A40007F018093F1000150110939F78C2FCF915C
:101A50001F910F91FF90EF9008958091F1020895EA
:101A60008091CA02811113C09FB7F8944091D603A8
:101A70005091D7036091D8037091D9039FBF443C24
:101A800059406105710518F081E08093CA020895FC
:101A9000EF92FF920F931F93CF93DF93D82F0FB640
:101AA00007FE46C080910503843079F080910301E0
:101AB00090E001962091050130E08223932320914C
:101AC00004012817190609F0C9C00E94300D8111C0
:101AD0000FC08091030190E001962091050130E054
:101AE00082239323209104012817190609F0B6C018
:101AF0000E947E078C01C091E900CF708091EC00BC
:101B000080FD37C080E0C82B83E08093E90085E04A
:101B1000E82E8091EB0085FD08C08091EB0080FFEE
:101B200004C08091EE0087FD44C0CF70C093E900EF
:101B3000E09103018E2F90E001962091050130E0A5
:101B400082239323209104012817190609F47EC0EB
:101B50008091010190910201E80FF92FF11DD083CE
:101B6000809103018F5F9091050189238093030188
:101B70006DC080E8C8CFE0910101F0910201E80F4B
:101B8000F11D90818F5F20910501822380930401D4
:101B90009093F1008091E80085FD0BC08091E800F2
:101BA00080FF07C08091E8008E778093E800E09284
:101BB00000018091040190910301981741F19091E7
:101BC000E80095FDD8CF80E029C01092F1002EC02A
:101BD0008091030190E001962091050130E082237D
:101BE0009323209104012817190609F09ECFF09045
:101BF0000001FF2009F499CF0E947E07801791070A
:101C000009F487CFFA94F09200018C0182CF809181
:101C1000E80085FFD8CFD093F10081E09091F200E9
:101C2000992379F09091E80090FF0BC09091E80023
:101C300095FDCBCF9091E8009E779093E800E092DD
:101C40000001882329F2CF70C093E90080E0DF9182
:101C5000CF911F910F91FF90EF900895E0910301B4
:101C600077CFEBECF2E011821082138212821582A0
:101C700014821782168211861086138612861586A4
:101C800014861786168608958330C9F128F48130AA
:101C900061F0823019F10895853009F452C008F4DA
:101CA0003FC0863009F45EC008958091170168171F
:101CB00090F4861B80931701809117011F928F93D8
:101CC00086E498E09F938F930E94DA050F900F901F
:101CD0000F900F90089510921701EECF809116018A
:101CE000681750F4861B80931601809116011F928D
:101CF0008F9384E398E0E6CF10921601F6CF80919F
:101D00001501681750F4861B809315018091150109
:101D10001F928F9381E298E0D5CF10921501F6CFF4
:101D200080911401681750F4861B809314018091F0
:101D300014011F928F938CE098E0C4CF109214018D
:101D4000F6CF80911301681750F4861B809313011E
:101D5000809113011F928F9383EF97E0B3CF10927E
:101D60001301F6CF80911201681750F4861B8093FF
:101D70001201809112011F928F9388ED97E0A2CFFC
:101D800010921201F6CF833009F445C028F4813057
:101D900061F0823049F10895853009F46AC008F491
:101DA00051C0863009F47CC0089580911701482FF6
:101DB000460F5527551F4F3F510594F4680F609308
:101DC0001701809117011F928F9389EC97E09F93E1
:101DD0008F930E94DA050F900F900F900F90089547
:101DE0008FEF80931701EDCF80911601482F460F9A
:101DF0005527551F4F3F510554F4680F6093160146
:101E0000809116011F928F9387EB97E0E0CF8FEFC1
:101E100080931601F5CF80911501482F460F552765
:101E2000551F4F3F510554F4680F60931501809181
:101E300015011F928F9384EA97E0C9CF8FEF8093AB
:101E40001501F5CF80911401482F460F5527551FD6
:101E50004F3F510554F4680F6093140180911401B1
:101E60001F928F938FE897E0B2CF8FEF809314018A
:101E7000F5CF80911301482F460F5527551F4F3F2F
:101E8000510554F4680F60931301809113011F9260
:101E90008F9386E797E09BCF8FEF80931301F5CF69
:101EA00080911201482F460F5527551F4F3F51056E
:101EB00054F4680F60931201809112011F928F9366
:101EC0008BE597E084CF8FEF80931201F5CFCF930E
:101ED000DF9320910803309109032817390701F196
:101EE0009093090380930803E091C703F091C8031E
:101EF0003097B1F0EC010084F185E02D09958091D7
:101F0000DC038570853061F4DF93CF938FED92E031
:101F10009F938F930E94DA050F900F900F900F9070
:101F2000DF91CF910895CF93DF93209106033091F5
:101F300007032817390701F19093070380930603DD
:101F4000E091C703F091C8033097B1F0EC0106802F
:101F5000F781E02D09958091DC038570853061F46F
:101F6000DF93CF9381ED92E09F938F930E94DA05E8
:101F70000F900F900F900F90DF91CF9108951F93C6
:101F8000CF93DF93E091C703F091C8033097E1F15D
:101F9000EC0118818091D103812B88830480F58125
:101FA000E02DCE01099518838091DC0383FF2CC0BE
:101FB0008C81282F082E000C330B3F938F938B813D
:101FC000282F082E000C330B3F938F938A81282FE4
:101FD000082E000C330B3F938F938981282F082EF6
:101FE000000C330B3F938F931F921F9386EB92E06D
:101FF0009F938F930E94DA058DB79EB70C960FB60C
:10200000F8949EBF0FBE8DBFDF91CF911F910895B1
:10201000CF93DF938091C8029091C902CFEFDFEF99
:102020009817D9F0E82FF0E0E853FE4F90818F5FCA
:102030008093C802C92FD0E01F929F9385E591E05D
:102040009F938F930E94DA050F900F900F900F903F
:10205000CF3FD10511F41092C701CE01DF91CF918E
:10206000089583EA98E00E9441051F9281E08F93D2
:102070001F9285E08F9385E598E09F938F930E9450
:10208000DA050F900F900F900F900F900F9008951A
:102090008091DC0383FF7EC08BE694E00E944105C3
:1020A0008091D1031F928F9386E694E09F938F9344
:1020B0000E94DA0584E694E00E9441058091D203F3
:1020C000282F082E000C330B3F938F9381E694E06A
:1020D0009F938F930E94DA058FE594E00E9441055B
:1020E0008091D303282F082E000C330B3F938F933E
:1020F0008CE594E09F938F930E94DA058AE594E043
:102100000E9441058091D403282F082E000C330B28
:102110003F938F9387E594E09F938F930E94DA0516
:1021200085E594E00E9441058091D503282F082E73
:10213000000C330B3F938F9382E594E09F938F9332
:102140000E94DA058FE494E00E9441058091CE035D
:102150001F928F938CE494E09F938F930E94DA05F3
:102160008AE494E00E9441058091CD031F928F93F1
:1021700087E494E09F938F930E94DA0584E494E0CF
:102180000E9441058DB79EB74C960FB6F8949EBF3E
:102190000FBE8DBF81ED93E00E94BF0F0E947E07AE
:1021A0009093D0038093CF0308950F931F93CF9301
:1021B000DF938091CB039091CA03892B8093BA015E
:1021C0009091C903992389F0892B8093BA01EBEB95
:1021D000F1E022EC31E080E0919191118F5F2E17B8
:1021E0003F07D1F781111092C903E091C703F09125
:1021F000C8033097B1F10280F381E02D8AEB91E0C2
:1022000009958091DC0382FF2CC080FF04C089EB1C
:1022100093E00E944105D0E0C0E003EB13E0809121
:10222000DC0380FF0EC0FE01E654FE4F80811F924A
:102230008F931F930F930E94DA050F900F900F90CA
:102240000F902196C830D10551F78091DC0380FFB3
:1022500008C081EB93E0DF91CF911F910F910C9417
:102260004105DF91CF911F910F9108951092CB03FB
:102270001092CA03EAEBF1E01182128213821482F7
:102280001582168217820E94D51085E0E1EDF3E0F9
:10229000DF011D928A95E9F71092CE031092CD03CB
:1022A0000E94481090E080E00E94930F90E080E050
:1022B0000C94670FCF93C82F1F928F938EE999E0EC
:1022C0009F938F930E94DA0581E090E0A0E0B0E058
:1022D00004C0880F991FAA1FBB1FCA95D2F780930D
:1022E000DD039093DE03A093DF03B093E0030F9030
:1022F0000F900F900F90CF910C943611882341F0DE
:1023000080959091CB0389238093CB030C94D510B7
:102310000895882339F09091CB03892B8093CB03C8
:102320000C94D51008958823E1F19CEF980F913A11
:1023300068F4EAEBF1E09281891301C012823196D0
:1023400041E0E03CF407B9F70C94D51090E2980F07
:10235000983088F4877021E030E0A90102C0440F72
:10236000551F8A95E2F7CA0180959091CB03892386
:102370008093CB03E9CF9BE5980F933020F490E056
:1023800080E00C94930F98E5980F973120F490E03B
:1023900080E00C94670F803F20F00E94E3050C94CE
:1023A000481008958732D8F58E3108F0FCC08E3081
:1023B00009F48FC078F4873009F470C08B3009F4C9
:1023C00056C0863009F458C088E495E00E94410563
:1023D00080E00895863109F4A6C078F48031A1F731
:1023E0009091DC03892F877F93FF88608093DC03C3
:1023F00083FF7FC087EE96E063C0893109F47CC01B
:102400008B3111F79091DC03892F8D7F91FF8260D2
:102410008093DC0381FF5AC080E297E051C088338B
:1024200031F150F4893221F0853311F0873261F6B1
:1024300080E00E945A1140C08334D1F320F48A33E3
:1024400018F28953F6CF883409F0BECF0E943611B6
:1024500086E497E00E9441052FEF83ED90E3215041
:1024600080409040E1F700C000000E9408098EE81B
:1024700094E00E94410520C08091DC03817F8E7F23
:102480008093DC0381E295E00E94410587E597E0B7
:102490000E94410581E08093DB0308958091DC0375
:1024A00080FF0CC089E397E00E9441058091DC0326
:1024B000817F8E7F8093DC0381E008958DE297E039
:1024C0000E9441058091DC038160F4CF82E197E0B6
:1024D000D0CF9091DC03892F8B7F92FF8460809313
:1024E000DC0382FF03C083E097E0EACF83EF96E04E
:1024F000C0CF8AED96E0BDCF8BEC96E00E944105FF
:102500008EE996E00E94410585E596E00E9441052E
:102510008FE296E00E9441058FED95E00E94410513
:1025200083EB95E0A6CF85EA95E00E9441050E94E5
:10253000E5081F928F938BE895E09F938F930E94FD
:10254000DA05809111011F928F9384E795E09F93A4
:102550008F930E94DA058091DA031F928F9381E6B0
:1025600095E09F938F930E94DA052FB7F89480919E
:10257000D6039091D703A091D803B091D9032FBF70
:10258000BF93AF939F938F938AE495E09F938F932C
:102590000E94DA058DB79EB742960FB6F8949EBF9B
:1025A0000FBE8DBF89CF8D5144CFCF93882309F4BF
:1025B000B1C0C82F8CEF8C0F813A08F057C18091C1
:1025C000DB03813071F1F8F0823009F45BC01092C6
:1025D000DB03ACEBB1E0EFEF80E09D91C91781F038
:1025E000EF3F19F4911101C0E82F8F5F8630A9F7F2
:1025F000EF3F31F00E2E000CFF0BE654FE4FC2836E
:10260000CF910C94D5108091BA01843421F0883890
:1026100011F08232F1F68C2F0E94D21181117AC012
:10262000D8CF8091BA018434B1F38838A1F38232D3
:1026300091F3C431C9F048F4CB3059F0C031C1F046
:102640008FEE92E00E94410511C0C93269F0C83393
:10265000B9F781E295E00E94410585EF92E00E9482
:10266000410581E08170DACF1092DB0380E0FACF80
:102670000E94311081EF92E00E94410582E0809338
:10268000DB03EFCFC432C8F4CE3108F0BEC0CB308C
:10269000E1F040F4C73009F4CFC08EE993E0CF9168
:1026A0000C944105C331C1F1C431B9F780910A03DB
:1026B000882349F110920A030AC0CB3409F4BAC046
:1026C000C0F4C93299F3C83341F70E9431108091A8
:1026D0000A03882309F4C7C01F928F9388E993E007
:1026E0009F938F930E94DA050F900F900F900F9099
:1026F00011C0C13509F498C0C23509F48FC0CE3479
:1027000061F66AE092C08DEA93E00E94410581E0A3
:102710008093DB03CF91089587E893E00E94410501
:1027200085E793E00E944105809117011F928F93E6
:1027300082E793E09F938F930E94DA0580E793E00E
:102740000E9441058EE593E00E94410580911601AB
:102750001F928F938BE593E09F938F930E94DA05EE
:1027600089E593E00E9441058AE493E00E944105D7
:10277000809115011F928F9387E493E09F938F932D
:102780000E94DA0585E493E00E94410584E393E02A
:102790000E944105809114011F928F9381E393E081
:1027A0009F938F930E94DA058FE293E00E94410588
:1027B0008AE193E00E944105809113011F928F935B
:1027C00087E193E09F938F930E94DA0585E193E080
:1027D0000E9441058EEF92E00E9441058091120116
:1027E0001F928F938BEF92E09F938F930E94DA0555
:1027F00089EF92E00E9441058DB79EB748960FB6CB
:10280000F8949EBF0FBE8DBF62CFCE51EC2FF0E08B
:10281000E85DFE4F808180930A0359CF61E080918B
:102820000A030E94C30E53CF61E080910A030E9405
:10283000440E4DCF6AE0F3CF8EE18093170182E31F
:10284000809316018AE08093150184E1809314013E
:1028500088E08093130188E28093120180EA93E07C
:102860000E94410534CF85E993E019CF80E28C0FB7
:10287000883068F4C77021E030E001C0220FCA95AB
:10288000EAF78091CB03822B8093CB03B9CE8BE503
:102890008C0F833068F481E890E0C53A31F083E82A
:1028A00090E0C63A11F482E890E0CF910C94930F37
:1028B00088E58C0F873108F068C082EE90E0C83A56
:1028C00009F460C089EE90E0C93A09F45BC08AEE71
:1028D00090E0CA3A09F456C085EB90E0CB3A09F48F
:1028E00051C086EB90E0CC3A09F44CC083EB90E009
:1028F000CD3A09F447C084EB90E0CE3A09F442C0E7
:1029000087EB90E0CF3AF1F18CEC90E0C13BD1F154
:102910008DEC90E0C03BB1F183E891E0C23B91F1D6
:102920008AE891E0C33B71F182E991E0C43B51F147
:1029300084E991E0C53B31F181E292E0C63B11F1BF
:1029400083E292E0C73BF1F084E292E0C83BD1F031
:1029500085E292E0C93BB1F086E292E0CA3B91F099
:1029600087E292E0CB3B71F08AE292E0CC3B51F0FF
:102970008FE690E0CD3B31F090E080E0CE3B11F46B
:1029800080E790E0CF910C94670FCF3B69F40E94F1
:1029900036119FEF20E782E0915020408040E1F720
:1029A00000C000000E940809C03F08F4B3CE8C2F7D
:1029B0000E94EE06CF910C944810CF92DF92EF92D6
:1029C000FF920F931F93CF93DF9300D000D01F92FD
:1029D000CDB7DEB76C0185E0F601DE0111960190FE
:1029E0000D928A95E1F7F60140815181238134816E
:1029F00091E02115310531F05F3F19F491E04F3F2F
:102A000009F090E090FD99C0F6010281F580F29402
:102A10009FE0F92249835A830B83722F3D832C83D5
:102A2000602F8D810E94A207182FE92FE295EF7089
:102A3000EF3008F082C0F0E0E05EFA4E0C9499228C
:102A40002F152F156D156D15E31515169D159D1573
:102A50002B169D15011701179D159D15BD17F92FF3
:102A6000FF70FF2E907F19F0F29480EFF822002380
:102A7000C9F0FF2039F08091CA03F82AF092CA0306
:102A80000E94D510812F0F900F900F900F900F90F4
:102A9000DF91CF911F910F91FF90EF90DF90CF903A
:102AA0000C94D512812F0E949311FF2009F445C088
:102AB000F0948091CA03F822F092CA030F900F900D
:102AC0000F900F900F90DF91CF911F910F91FF907A
:102AD000EF90DF90CF900C94D510892F8F70907F5E
:102AE000903211F08295807F112379F0113009F432
:102AF00049C0002309F455C0FF2059F0F601958123
:102B000090FF8DC19F70958304C0002321F1F110C7
:102B10000FC00F900F900F900F900F90DF91CF91FB
:102B20001F910F91FF90EF90DF90CF900C9489113F
:102B300021E0F212EECF8093C9030F900F900F9017
:102B40000F900F90DF91CF911F910F91FF90EF9019
:102B5000DF90CF900895F11011C01092C9030F902B
:102B60000F900F900F900F90DF91CF911F910F91C9
:102B7000FF90EF90DF90CF900C947E1191E0F912CE
:102B8000ECCFDBCF002349F0E5E0EF15B0F29091F8
:102B9000CB03982309F4BDCFE2CFF4E0FF1568F230
:102BA000DECFFF20E1F2812F0F900F900F900F905A
:102BB0000F90DF91CF911F910F91FF90EF90DF90D9
:102BC000CF900C949311892F869586958370C1F0D0
:102BD000813009F0B2CF812F9370011102C090E0D3
:102BE00080E00F900F900F900F900F90DF91CF919A
:102BF0001F910F91FF90EF90DF90CF900C94670F93
:102C0000812F9370011102C090E080E00F900F902F
:102C10000F900F900F90DF91CF911F910F91FF9028
:102C2000EF90DF90CF900C94930F002389F00E94D7
:102C3000EE060F900F900F900F900F90DF91CF91B5
:102C40001F910F91FF90EF90DF90CF900C94481060
:102C50000E94E305EECF892F837009F064C0011153
:102C60006CCF812F829586958770880F880F412FB2
:102C70004F70C42ED12CF12CE12C082E04C0CC0CAA
:102C8000DD1CEE1CFF1C0A94D2F740E050E0BA01B4
:102C900014FF11C00FE010E020E030E004C0000F8E
:102CA000111F221F331F8A95D2F7B901A801409541
:102CB0005095609570950091DD031091DE03209191
:102CC000DF033091E0039695969593709230E9F08A
:102CD00028F5913089F04C295D296E297F29402300
:102CE0005123622373234093DD035093DE036093EB
:102CF000DF037093E00321CFC02AD12AE22AF32A0E
:102D00004C295D296E297F29EECF4C295D296E293A
:102D10007F294027512762277327E5CF402351237E
:102D200062237323EDCF8695002311F0892F8170E4
:102D3000882309F402CF812F829586958770880FAA
:102D4000880F412F4F70C42ED12CF12CE12C082E6E
:102D500004C0CC0CDD1CEE1CFF1C0A94D2F740E032
:102D600050E0BA0114FF11C00FE010E020E030E0A5
:102D700004C0000F111F221F331F8A95D2F7B9011B
:102D8000A80140955095609570950091430310916E
:102D90004403209145033091460396959695937090
:102DA0009230E9F028F5913089F04C295D296E299F
:102DB0007F2940235123622373234093430350937D
:102DC00044036093450370934603B7CE0C291D2935
:102DD0002E293F29402B512B622B732BEECF4C29F0
:102DE0005D296E297F294027512762277327E5CF68
:102DF00040235123622373234C295D296E297F29A7
:102E0000DCCF803F09F44EC0D0F480E4810F8032E3
:102E100070F1002309F4ACC0FF2009F4A6C0812F93
:102E20000E94D512193309F099C0FFEF21EE84E01A
:102E3000F15020408040E1F700C000007ECE823F8C
:102E400009F470C008F45BC0833F19F7002309F44C
:102E50007CC0292F2F7181E090E0A0E0B0E004C099
:102E6000880F991FAA1FBB1F2A95D2F73AC0E12FDE
:102E7000E071FE2E892F8F71002351F00E946F08A0
:102E8000812F8295807FF11044CE812F8F7041CEAB
:102E90000E944B08812F8295807FF11060CE812F98
:102EA0008F705DCE002331F1F4E0FF1508F445CEBC
:102EB000292F2F7181E090E0A0E0B0E004C0880FDE
:102EC000991FAA1FBB1F2A95D2F740914303509127
:102ED0004403609145037091460384279527A627F4
:102EE000B7278093430390934403A0934503B09383
:102EF000460323CE25E02F1508F41FCED9CF892F06
:102F00008F71002399F00F900F900F900F900F90FA
:102F1000DF91CF911F910F91FF90EF90DF90CF90B5
:102F20000C946F08892F8F71002369F30F900F9015
:102F30000F900F900F90DF91CF911F910F91FF9005
:102F4000EF90DF90CF900C944B08109243031092B7
:102F500044031092450310924603EFCD133509F454
:102F600064CF173409F0E9CD60CF892F8F71CBCFB3
:102F7000F11019CE892F8F71D9CF8111DECD0023A9
:102F800009F4DBCD0E9436118FEF90E7E2E081502B
:102F90009040E040E1F700C000000E9408091F9344
:102FA000CF93DF9380911003807FB1F480910D0364
:102FB000882391F02091420310911103C0910B03DB
:102FC000D0910C03A0910E03B0910F0341E0CF3FCD
:102FD00009F040E0121304C0DF91CF911F910895D2
:102FE00081E0109721F0842FDF3F09F080E030E08E
:102FF00080FD33C0C90166E070E00E947422FC01CC
:10300000EE5EFC4F81818D1328C080818C1325C01A
:103010008281811122C0838194818A1B9B0B883C11
:103020009105D8F4809110038F7080618093100314
:10303000C90166E070E00E947422FC01E95EFC4F69
:1030400090819F70906190838BE093E00E94DD14EB
:10305000DF91CF911F910C948F082F5F3F4F277006
:10306000B9CF9F92AF92BF92CF92DF92EF92FF9231
:103070000F931F93CF93DF93CDB7DEB761970FB652
:10308000F894DEBF0FBECDBF8C0185E0F801DE01F4
:103090001D9601900D928A95E1F7F80140812181FA
:1030A000F280C380D48090910B0330910C03609127
:1030B0000E0370910F0381E06115710531F03F3F00
:1030C00019F481E09F3F09F080E0F82FF1709F2E06
:1030D00080FD4EC18BE0A82E83E0B82EE0900D035A
:1030E000F601E61BF70BEE2009F404C180911003F2
:1030F000582F507FE83CF10508F0BDC0511183C046
:10310000EF2C321322C0941320C0F1101EC08F7018
:10311000806180931003C5010E94DD14809110032B
:10312000F80185838E2D61960FB6F894DEBF0FBE31
:10313000CDBFDF91CF911F910F91FF90EF90DF9066
:10314000CF90BF90AF909F90089581E0C114D104BB
:1031500031F02F3F19F481E04F3F09F080E080FD0E
:1031600014C081E08F25F82FF170BF2EE09142034B
:103170003091110380FD22C0FF20A1F28091100345
:10318000816080931003E12CCDCF80E0ECCFF0E0A4
:10319000CF0166E070E00E947422DC01AE5EBC4F9D
:1031A00011968C911197281307C08C91481304C075
:1031B00012968C918F11E0CF3196E770E313E7CF31
:1031C0007C2DD98AC88A522F6F2D89890E94A20727
:1031D000292F22952F70223050F0243078F49F70E0
:1031E00051F0F8019581907F31F4E92C9BCF9F70CD
:1031F00011F08823D1F3805E8830B8F3C8010E94B3
:10320000DD149B2CF2CF321306C0941304C0F801D6
:10321000FF2009F48AC04D872E87FF867C2DD98A2E
:10322000C88A522F6F2D89890E949908882309F432
:10323000AEC0FF2009F4ABC080911003803270F063
:1032400020910B0330910C0338872F831986DB867E
:10325000CA868C87CE0107960E94DD1486E0F801AD
:10326000ABE0B3E001900D928A95E1F70E94CF1791
:10327000EE24E39457CF51110AC08BE093E00E94F3
:10328000DD1486E0F50111928A95E9F77CCF3213BF
:103290000FC094130DC0F1100BC0F8018583C80155
:1032A0000E94DD1486E0F50111928A95E9F73ACF84
:1032B0004D872E87FF867C2DD98AC88A522F6F2D85
:1032C00089890E949908882309F461C0FF2009F4C4
:1032D0005EC080911003803208F220910B03309180
:1032E0000C033A8329831B82DD82CC828E83CE013C
:1032F0000196B2CFE83CF105A8F6EF2CFF2009F4C7
:1033000046C032131FC094131DC08091100380FD6E
:1033100010C0982F907F69F0F8018583903F31F0BD
:10332000982F907F905F8F70892B8583C8010E94B2
:10333000DD1486E0F801ABE0B3E001900D928A95D0
:10334000E1F7F0CE4D872E87FF867C2DD98AC88A7B
:10335000522F6F2D89890E94990881117FCF80910A
:103360001003816080931003C8010E94DD14DACE3F
:10337000FF2069F04D872E87FF867C2DD98AC88A69
:10338000522F6F2D89890E949908811167CFC8013A
:103390000E94DD146DCFCF93DF93CDB7DEB7679773
:1033A0000FB6F894DEBF0FBECDBF4B8B5C8B6D8B21
:1033B0007E8B8F8B1A8A198A85E0FE017396DE0157
:1033C0001D9601900D928A95E1F786E0FE013D96EB
:1033D000DE01179601900D928A95E1F7CE010796CE
:1033E0000E943118811138C086E0FE013796DE0157
:1033F000119601900D928A95E1F79F8188852A8523
:103400003B85232B39F08F3F19F481E09F3F19F062
:1034100080E001C081E080FD1FC08091110390E039
:103420009C012F5F3F4F2770332740914203421783
:10343000130661F166E070E00E947422DC01AE5E6A
:10344000BC4F96E0FE01319601900D929A95E1F7FE
:10345000209311030E948F088091420390911103E1
:10346000891709F190E066E070E00E9474228E5E98
:103470009C4F0E9431188823B1F08091420390E064
:1034800001968770992780934203E6CF0E943611F8
:10349000109211031092420386E0EBE0F3E0DF01AB
:1034A0001D928A95E9F767960FB6F894DEBF0FBEB6
:1034B000CDBFDF91CF910895CF93DF9300D01F92BE
:1034C000CDB7DEB720910503243041F520911001DE
:1034D000222321F123E029839B838A8382E0809346
:1034E000E9008FEF9091E800815095FD06C095EDC1
:1034F0009A95F1F700008111F5CF8091E80085FFE2
:103500000DC050E040E063E070E0CE0101960E9403
:10351000010D8091E8008E778093E8000F900F9066
:103520000F90DF91CF910895CF93DF9300D01F923A
:10353000CDB7DEB720910503243081F5209110012D
:10354000222361F119821A821B8222E029838138A9
:10355000910520F0805891099B838A8382E08093B3
:10356000E9008FEF9091E800815095FD06C095ED40
:103570009A95F1F700008111F5CF8091E80085FF61
:103580000DC050E040E063E070E0CE0101960E9483
:10359000010D8091E8008E778093E8000F900F90E6
:1035A0000F90DF91CF91089520910503243049F5C4
:1035B00022E02093E9002FEF3091E800215035FD03
:1035C00006C035ED3A95F1F700002111F5CF2091B5
:1035D000E80025FF16C02091100150E040E063E0B4
:1035E00070E0222339F021E02093F10050E040E028
:1035F00065E070E00E94010D8091E8008E77809375
:10360000E8000895CF93DF9320910503243011F54E
:1036100021E02093E90021E8215021F03091E800D9
:1036200035FF1BC02091E80025FF14C0EC0150E0DD
:1036300040E068E070E00E94010D8091E8008E7724
:103640008093E80088E0FE01A2EFB2E001900D92C5
:103650008A95E1F7DF91CF910895EFE3F1E031979B
:10366000F1F700C00000D8CFCF93C82F1F928F93DF
:103670008CE591E09F938F930E94DA053FB7F89411
:103680005B9A45EA4A95F1F700000F900F900F9072
:103690000F9088E090E021E04C2F422381F05B986E
:1036A00045EA4A95F1F70000220F0197A9F75B98C8
:1036B00085EA8A95F1F700003FBFCF9108955B9AA4
:1036C000EFCFCF93DF9300D000D01F92CDB7DEB7FE
:1036D0008091C701813009F44FC078F0823009F43D
:1036E00090C0833009F432C180E00F900F900F90AA
:1036F0000F900F90DF91CF9108950E9408108FEFE7
:103700000E94341B8FE99FE00197F1F700C0000091
:103710000E9408108F3F910551F09FEFA3EDB0E399
:103720009150A040B040E1F700C00000DDCF8EEF27
:103730000E94341B8FE99FE00197F1F700C0000061
:103740000E9408108E3F910541F78DEF0E94341BB7
:10375000AFE9BFE01197F1F700C000000E94081028
:103760008D3F9105D1F683E30E94341B0E9408101F
:1037700081E08093C701B8CF0E940810803891057E
:103780003CF497FF35C00196E1F01092C701ACCF31
:103790009C01205C310920323105B8F744E0880FE4
:1037A000991F4A95E1F780778093C501AFE8B1E0B2
:1037B0001197F1F700C000008FE30E94341B82E0F4
:1037C000D8CF9091DB028091C601981709F48CCF75
:1037D0008FE99FE00197F1F700C000008091DB02C4
:1037E00087700E94341B8091DB028093C6017CCFDE
:1037F00086FD80688093C4018FE30E94341B83E0C0
:10380000B8CF0E9408108F3FBFEF9B0709F46CCF21
:103810000CF4BBCF9C01205C31092032310508F04B
:10382000B4CF282F2F703091C501232B807D99278D
:10383000803D910509F441C02093C5018FE891E0D6
:103840000197F1F700C0000083E30E94341B81E080
:103850008093C7018091C50187FF4FC0982F9F7744
:103860009057933060F5837021E030E0D90102C0B9
:10387000AA0FBB1F8A95E2F7CD0180959091C301F5
:1038800098239093C301FE01319685E0DF011D92DC
:103890008A95E9F79983CF010E94BF0F8091C501F6
:1038A0001F928F9381E791E09F938F930E94DA0597
:1038B0000F900F900F900F9017CF2068BDCFE82F7B
:1038C000F0E033E0F695E7953A95E1F7EE70FF27E3
:1038D000E553FD4F8F7021E030E0A90102C0440F95
:1038E000551F8A95E2F7CA01809590952081318114
:1038F0008223932391838083D1CF90E9980F9330D3
:1039000058F4837021E030E001C0220F8A95EAF775
:103910009091C301922BB5CFE82FF0E094E0F5959C
:10392000E7959A95E1F7EE0FFF1FE553FD4F8F7076
:1039300021E030E0A90102C0440F551F8A95E2F74B
:10394000CA0120813181822B932BD4CF0E94081091
:103950008F3F5FEF950709F4C7CE0CF416CF803880
:1039600091050CF012CF86FD80688093C201082E6D
:10397000000C990B9F938F938091C401282F082EE0
:10398000000C330B3F938F9383E691E09F938F93CB
:103990000E94DA051B821C821D828091C3018983EB
:1039A0008091C4018A838091C2018B83CE010196EC
:1039B0000E94BF0F8FE891E00197F1F700C000006F
:1039C00083E30E94341B81E08093C7010F900F9026
:1039D0000F900F900F900F9087CE78941F920F92B8
:1039E0000FB60F9211248F939F93AF93BF93809143
:1039F000D6039091D703A091D803B091D903019633
:103A0000A11DB11D8093D6039093D703A093D80333
:103A1000B093D903BF91AF919F918F910F900FBE3B
:103A20000F901F9018951F920F920FB60F921124AE
:103A30008F939F93AF93BF938091CC03811113C059
:103A40008091D6039091D703A091D803B091D90368
:103A50004196A11DB11D8093D6039093D703A093E7
:103A6000D803B093D903BF91AF919F918F910F90DD
:103A70000FBE0F901F9018951F920F920FB60F92C6
:103A800011242F933F934F935F936F937F938F9363
:103A90009F93AF93BF93EF93FF938091E10082FFD9
:103AA00009C08091E20082FF05C08091E1008B7F18
:103AB0008093E1008091E10080FF21C08091E200CD
:103AC00080FF1DC08091E2008E7F8093E200809194
:103AD000E20080618093E2008091D8008062809350
:103AE000D80019BC85E0809305038091F102809392
:103AF000F0021092F1020E94310E0E943611809164
:103B0000E10084FF2FC08091E20084FF2BC084E09D
:103B100089BD86E089BD09B400FEFDCF8091D80043
:103B20008F7D8093D8008091E1008F7E8093E100AB
:103B30008091E2008F7E8093E2008091E2008160BC
:103B40008093E2008091FC02882309F460C084E045
:103B5000809305030E94310E0E9436118091F0027D
:103B60008093F1028091E10083FF40C08091E200E8
:103B700083FF3CC08091E100877F8093E10082E079
:103B8000809305031092FC028091E1008E7F809368
:103B9000E1008091E2008E7F8093E2008091E2005C
:103BA00080618093E20042E060E080E00E94D10901
:103BB00081E0809311011092DA031092F10298E0F3
:103BC000E2EFF2E0DF011D929A95E9F71092BB0156
:103BD0001092BC011092BD011092BE011092BF0163
:103BE0001092C0011092C10180931001FF91EF91DA
:103BF000BF91AF919F918F917F916F915F914F9105
:103C00003F912F910F900FBE0F901F9018958091AC
:103C1000E30087FD02C081E09BCF83E099CFCF9383
:103C2000DF93CDB7DEB72B970FB6F894DEBF0FBE8C
:103C3000CDBF84B7877F84BF0FB6F894A8958091D5
:103C40006000886180936000109260000FBE80E881
:103C500090E00FB6F89480936100909361000FBEDE
:103C600088E49DE0909339018093380186E091E0EB
:103C70009093C8038093C7038BEE91E00E944105A7
:103C80000E94F108809163008E7F8093630081E041
:103C90008093EF021092E2001092E1008091D80030
:103CA0008F778093D8008091D80080688093D80067
:103CB0008091D8008F7D8093D80084E089BD86E014
:103CC00089BD09B400FEFDCF109205031092FC02DD
:103CD0001092FB021092FA0242E060E080E00E9443
:103CE000D1098091E1008E7F8093E1008091E20014
:103CF00081608093E2008091E20088608093E2001E
:103D00008091E0008E7F8093E000789482E084BD13
:103D100093E095BD9AEF97BD80936E000E94310E9F
:103D2000529A5198599A809169008C6080936900E9
:103D3000E99A7894539A5B988AE791E00E9441054A
:103D400080910503843009F04AC10E94300D882318
:103D500009F445C189ED91E00E9441058BEC91E0A9
:103D60000E94410548E1242E41E0342E8091050354
:103D7000853009F437C10E94611B0DED12E03BEC68
:103D8000432E32E0532E912CF201A190B1902F01DD
:103D9000F801C080D180CA14DB0409F461C08091AD
:103DA000DC0381FF2FC08AE991E00E9441052BECE2
:103DB000622E22E0722EF12CE12CF3018081F18140
:103DC000FB8722E0620E711C0E948A07882E8B8579
:103DD0000E948A073F922F928F928F93FF92EF92C9
:103DE0008EE891E09F938F930E94DA05FFEFEF1A20
:103DF000FF0A0FB6F894DEBF0FBECDBF98E0E916FC
:103E0000F104D9F6812CEE24E394F12CCA24DB24AE
:103E1000C6018E219F21892BE9F08E829F8221E0AD
:103E2000C7018A219B21892B09F420E028870E9461
:103E30007E078160782F9A8789874E815F816885A8
:103E40008A850E94CB19F801808191818E259F255A
:103E5000918380838394EE0CFF1CF0E18F12D8CF06
:103E600093940E5F1F4F28E092128ECF8FEF8983BD
:103E70008A831B820E947E078160782F9D838C83BA
:103E800049815A816B818D810E94CB198091CF032A
:103E90009091D0032FB7F8944091D6035091D70357
:103EA0006091D8037091D9032FBFFA01E81BF90B79
:103EB0002091CE038091160190E0211107C08091DE
:103EC000170190E06AE070E00E947422E817F90799
:103ED00080F08091D203F090D3031091D40300912D
:103EE000D5038111BBC0F1107FC111117DC101113A
:103EF0007BC10E94E5089091DC028917D9F10E94EC
:103F0000E5088093DC029091DC039570953061F4B4
:103F10001F928F9380EC91E09F938F930E94DA051C
:103F20000F900F900F900F908091DC0280FD04C1E4
:103F30001092DB0281FF05C09091DB0291609093AB
:103F4000DB0282FF05C09091DB0294609093DB025C
:103F50009091DB021F929F931F928F938FEA91E0C3
:103F60009F938F930E94DA050F900F900F900F9000
:103F70000F900F902091E4003091E5008091ED02C8
:103F80009091EE022817390739F18091E400909161
:103F9000E5009093EE028093ED020E94300D88239D
:103FA000D9F0809105038430B9F48091E9008F70D5
:103FB0009091EC0090FFC4C090E8892B93E090931F
:103FC000E9009091EB0090FF04C09091EE0097FD06
:103FD000D5C08F708093E9000E94030AC7CE0E946B
:103FE000030AAECE80910503843021F11092CC03F8
:103FF00088E190E020E40FB6F894A89580936000E3
:104000000FBE2093600083B7817F846083BF83B736
:10401000816083BF7894889583B78E7F83BF0FB606
:10402000F894A89580916000886180936000109258
:1040300060000FBE8091FB02882309F497CE0E9496
:10404000611BEBECF2E081919191892B09F0B6C0F4
:104050008BED92E08E179F07B1F788CE2F3F19F0B6
:104060002F5F2093CE03181624F40E94A20680939B
:10407000D2038091D20387FF05C00E94A2068195DA
:104080008093D2031F1424F40E94A2068093D303CA
:104090008091D30387FF05C00E94A206819580937B
:1040A000D3036091D203662331F1F090D303FF2054
:1040B00011F1062E000C770B880B990B0E947321CF
:1040C00023E333E343E35FE30E94D7210E943B21D4
:1040D0006093D2036F2DFF0C770B880B990B0E9416
:1040E000732123E333E343E35FE30E94D7210E947C
:1040F0003B216093D303111624F40E94670680933A
:10410000D4038091D40387FF05C00E946706819580
:104110008093D403101624F40E9467068093D5037D
:104120008091D50387FF05C00E9467068195809323
:10413000D5030E944810DDCE92E09093DB02FACEC8
:1041400090E03BCFE0910101F0910201E90FF11DF8
:1041500020819F5F30910501932390930401209368
:10416000F1009091E80095FD09C09091E80090FF62
:1041700005C09091E8009E779093E800909104012B
:1041800020910301291721F02091E80025FDDACFC5
:104190009091F200992309F41CCF9091E80090FFD0
:1041A00018CF9091E80095FD06C09091E8009E77A9
:1041B0009093E8000ECF1092F100F3CF84E089BD18
:1041C00086E089BD09B400FEFDCF8091D8008F7DC7
:1041D0008093D8008091E00082608093E00080911D
:1041E000E00081FDFCCFC2CD2F3F09F039CF4ACF8F
:1041F0001F920F920FB60F9211242F933F934F935C
:104200008F939F93EF93FF934A9A499B28C040E571
:104210004A95F1F74A9A28E030E081E090E045EADB
:104220004A95F1F700004A9A499B982B880F215034
:104230003109A9F785EA8A95F1F700008091C90252
:10424000E82FF0E08F5F2091C802281729F0E8538B
:10425000FE4F90838093C90282E08CBB4A9AFF9103
:10426000EF919F918F914F913F912F910F900FBEA2
:104270000F901F9018950E9442216894B1110C94E0
:10428000D12108950E94B62188F09F5798F0B92F48
:104290009927B751B0F0E1F0660F771F881F991F7B
:1042A0001AF0BA95C9F714C0B13091F00E94D0212C
:1042B000B1E008950C94D021672F782F8827B85F3C
:1042C00039F0B93FCCF3869577956795B395D9F7D3
:1042D0003EF490958095709561957F4F8F4F9F4FDD
:1042E0000895E89409C097FB3EF4909580957095E9
:1042F00061957F4F8F4F9F4F9923A9F0F92F96E932
:10430000BB279395F695879577956795B795F111A6
:10431000F8CFFAF4BB0F11F460FF1BC06F5F7F4F43
:104320008F4F9F4F16C0882311F096E911C0772355
:1043300021F09EE8872F762F05C0662371F096E85E
:10434000862F70E060E02AF09A95660F771F881F2D
:10435000DAF7880F9695879597F9089557FD905845
:10436000440F551F59F05F3F71F04795880F97FB39
:10437000991F61F09F3F79F08795089512161306F3
:104380001406551FF2CF4695F1DF08C01616170622
:104390001806991FF1CF8695710561050894089557
:1043A000E894BB2766277727CB0197F908950E94E9
:1043B000E9210C9463220E94552238F00E945C226D
:1043C00020F0952311F00C944C220C9452220C9462
:1043D000D1210E94AE2178F39923C9F35523B9F373
:1043E000950F50E0551FAA27EE27FF27BB27002473
:1043F0000894679520F4E20FF31FB41F0A1E220FE2
:10440000331F441FAA1F6695A9F7779530F4F30F61
:10441000B41F0A1E121E08F46395330F441FAA1F0F
:10442000221F769599F7879520F4B40F0A1E121E65
:10443000631F440FAA1F221F331F8695A9F7862FDB
:10444000712D602D11249F5750409AF0F1F0882370
:104450004AF0EE0FFF1FBB1F661F771F881F91508A
:104460005040A9F79E3F510580F00C944C220C94CB
:10447000D1215F3FE4F3983ED4F386957795679515
:10448000B795F795E7959F5FC1F7FE2B880F911DB4
:104490009695879597F9089597F99F6780E870E05A
:1044A00060E008959FEF80EC089500240A941616AA
:1044B000170618060906089500240A941216130612
:1044C000140605060895092E0394000C11F48823A0
:1044D00052F0BB0F40F4BF2B11F460FF04C06F5FBC
:1044E0007F4F8F4F9F4F08950024552704C0080E1B
:1044F000591F880F991F009729F076956795B8F393
:104500007105B9F7802D952F089597FB072E16F4A6
:10451000009407D077FD09D00E949F2207FC05D0A8
:104520003EF4909581959F4F0895709561957F4FCA
:104530000895EE0FFF1F0590F491E02D0994AA1B3A
:10454000BB1B51E107C0AA1FBB1FA617B70710F07E
:10455000A61BB70B881F991F5A95A9F780959095B0
:0A456000BC01CD010895F894FFCFCF
:10456A00053A0100007F2D0D021BD41A941A5C1A19
:10457A0001012808140A321E00407F221501960004
:10458A00740016022F0248020102030405060708F6
:08459A00090000080004000202
:106800008800EA44E944E244040005000600070069
:10681000080009000A000B000C000D000E000F001C
:1068200010001100120013001400150016001700CC
:10683000180019001A001B001C001D001E001F007C
:10684000200021002200230024002500260027002C
:10685000280029002A002B002C002D002E002F00DC
:10686000300031003200330034003500360037008C
:10687000380039003A003B003C003D003E003F003C
:1068800040004100420043004400450046004700EC
:10689000480049004A004B004C004D004E004F009C
:1068A000500051005200530054005500560057004C
:1068B000580059005A005B005C005D005E005F00FC
:1068C000600061006200630064006500850067008D
:1068D000680069006A006B006C006D006E006F005C
:1068E0007000710072007300890087008A008B00BD
:1068F000E000E100E200E300F1A1E500E600E700CE
:106900000100010001000100EA4401000100E2442D
:106910000100010001000100460001004A004B0097
:10692000010001004700480001000100E9440100A6
:106930000100010001000100010001003A003B00DC
:106940003C003D003E003F0040004100420043004B
:10695000010035004C0039000100440045005200A0
:1069600049000100010050004F0029004D004E0079
:1069700051000100010001000100010001000100BF
:1069800001000100010001000100010001000100FF
:1069900001000100010001000100010001004D00A3
:1069A0004A004E004B0001000100010001000100FF
:1069B000F6000100F1000100F2000100F300010007
:1069C000F0000100F400F5000100010001000100E9
:1069D00001000100010001000100010001000100AF
:1069E0000100010001000100490001000100010057
:1069F000010001000100010001000100010001008F
:00000001FF
